:100000000C9475060C94BC060C94BC060C94BC06AF
:100010000C94BC060C94BC060C94BC060C94BC0658
:100020000C94BC060C94BC060C94A1150C9473168D
:100030000C9406250C94BC060C94BC060C94BC06CF
:100040000C94BC060C94BC060C94BC060C94BC0628
:100050000C94BC060C94A6250C94BC060C94BC060F
:100060000C94BC060C9418090C94BC060C94BC06A9
:100070000C94BC060C94BC060C94BC060C94BC06F8
:100080000C94BC060C94BC060C94BC060C94BC06E8
:100090000C94BC060C94BC060C94BC060C94BC06D8
:1000A0000C94BC060C94BC060C94BC06440E480E82
:1000B0004C0E500E540E580E5C0E600E640E680E00
:1000C0006C0E700E740E780E7C0E800E840E880EF0
:1000D0008C0E900E940E980E9C0EA00EA40EA80EE0
:1000E000AC0EB00EB40EB80EBC0EC00EC40EC80ED0
:1000F000CC0ED00E100F420ED40ED60ED80EDA0E45
:10010000DE0EE20EE60EEA0EEF0EF40EF80EFC0E18
:10011000000F040F080F0E0F0E0F0E0F0E0F0E0F15
:100120000E0F0E0F0E0F0E0F0E0F0E0F0E0F0E0FE7
:100130000E0F0E0F0E0F0E0F0E0F0E0F0C0FE01600
:100140000217F0170217F01747176A17F017BF17B3
:10015000D217FA1AFA1A291B291B871BC51BDF1D88
:10016000DF1DDE1BDF1DDF1CDF1CB31DDF1DDF1DE0
:10017000CA1D8080352B78793980808021087706E8
:1001800007808080201A7A1B168080801E8029803C
:10019000808080808080808080808080221580198F
:1001A000098080801F147B1D0480808023172C050C
:1001B0000A808080260C00360E80808025187610FC
:1001C0000D808080241C80110B80808027127E3758
:1001D0000F8080802A804F7D28808080743051522B
:1001E000328080802D137C38338080802E2F507594
:1001F000348025630025730D0A00522C310D0A004E
:1002000053592C464646340D0A0053482C3030339F
:10021000430D0A00537E2C360D0A0053572C3830FC
:1002200030300D0A00534D2C340D0A0053532C4B23
:100230006579626F6172642F4D6F7573650D0A0089
:10024000532D2C546D6B42540D0A0053462C310D26
:100250000A002D2D2D0D0A0045786974696E6720FE
:10026000636F6E666967206D6F6465202E2E2E0A9F
:10027000002B0D0A00760D0A0024242400456E741C
:100280006572696E6720636F6E666967206D6F6463
:1002900065202E2E2E0A00522C310D0A0053522CAE
:1002A0005A0D0A00555342206D6F64650A0041756E
:1002B000746F206D6F64650A00253032750A002561
:1002C0003032753A00253032753A004241543A20B6
:1002D00025756D560900757074696D653A20253075
:1002E000327520253032753A253032753A25303254
:1002F000750A00564255533A2025580A0052656D3A
:100300006F746557616B657570456E61626C65648D
:100310003A2025580A000A003F004C4F5700444934
:10032000534348470043484152470046554C4C0010
:10033000626174746572793A200055534220537497
:100340006174653A2025730A00636F6E6669675FA2
:100350006D6F64653A2025580A00726E34325F6111
:1003600075746F636F6E6E656374696E6728293A82
:100370002025580A00726E34323A2025730A00662E
:100380006F7263655F7573623A2025580A00707258
:100390006F746F636F6C3A2025730A000A2D2D2D40
:1003A0002D2D20524E2D343220696E666F202D2D5A
:1003B0002D2D2D0A00753A20202020202020746F3A
:1003C00067676C6520466F72636520555342206DE8
:1003D0006F64650A00703A20202020202020706180
:1003E0006972696E670A00536C636B3A20202020A3
:1003F000524E2D343220696E697469616C697A6578
:100400000A0044656C3A2020202020656E746572D5
:100410002F6578697420524E2D343220636F6E66DA
:100420006967206D6F64650A00623A2020202020F1
:1004300020206261747465727920766F6C746167D4
:10044000650A00693A20202020202020524E2D34B9
:100450003220696E666F0A000A0A2D2D2D2D2D207F
:10046000426C7565746F6F746820524E2D34322063
:1004700048656C70202D2D2D2D2D0A0025303275EC
:100480003A253032753A253032750925756D560A90
:10049000004C4544207374617475733A20253032E2
:1004A000580A002025303258002563005B735D0038
:1004B0004B6579626F6172642073746172740A00B3
:1004C000524E2D343220696E69740A000A55534227
:1004D00020696E69740A005B445D005B435D001235
:1004E00003480048004B00420020006D006F00648C
:1004F0000000000E0374002E006D002E006B002E15
:100500000000000403090409027400040100A03281
:100510000904000001030101000921110100012269
:1005200040000705810308000A09040100010301D6
:100530000200092111010001224D00070582030874
:10054000000A090402000103000000092111010052
:10055000012236000705830308000A09040300028C
:100560000300000009211101000122220007058477
:1005700003200001070504032000011201100100FF
:10058000000008EDFE42420401010200010631FFB5
:100590000974A1010975150026FF009520750881D1
:1005A000020976150026FF00952075089102C00506
:1005B000010980A101850216810026B7001A810079
:1005C0002AB700751095018100C0050C0901A10131
:1005D0008503160100269C021A01002A9C02751050
:1005E00095018100C005010902A1010901A10005D1
:1005F0000919012905150025019505750181029547
:1006000001750381010501093009311581257F95A7
:10061000027508810609381581257F9501750881C5
:1006200006050C0A38021581257F9501750881069B
:10063000C0C005010906A101050719E029E7150059
:10064000250195087501810295017508810105084C
:10065000190129059505750191029501750391010F
:100660000507190029FF150026FF0095067508816A
:1006700000C0636F6E73756D65723A202530345813
:100680000A0073797374656D3A20253034580A0076
:100690000A002530325820006B6579626F61726400
:1006A0003A20004C45443A20253032580A00253083
:1006B00032583A202530386225730A00722F6320A1
:1006C00030313233343536370A004F6E6573686F18
:1006D000743A2074696D656F75740A00290A0025E3
:1006E00075002F002575005D280025640020002579
:1006F0006400200025640020002564007C00253073
:100700003258006D6F7573656B6579205B62746E2E
:100710007C782079207620685D287265702F61636F
:100720006C293A205B006D6B5F776865656C5F7460
:10073000696D655F746F5F6D6178203D2025640A87
:10074000006D6B5F776865656C5F6D61785F737076
:10075000656564203D2025640A006D6B5F74696DDA
:10076000655F746F5F6D6178203D2025640A006DC0
:100770006B5F6D61785F7370656564203D202564F3
:100780000A006D6B5F696E74657276616C203D2046
:1007900025640A006D6B5F64656C6179203D2025DE
:1007A000640A006D6B5F776865656C5F74696D6581
:1007B0005F746F5F6D6178203D2025640A006D6B6A
:1007C0005F776865656C5F6D61785F7370656564A0
:1007D000203D2025640A006D6B5F74696D655F7450
:1007E0006F5F6D6178203D2025640A006D6B5F6D41
:1007F00061785F7370656564203D2025640A006D33
:100800006B5F696E74657276616C203D2025640AA9
:10081000006D6B5F64656C6179203D2025640A0082
:100820000A00257500363A20776865656C5F746943
:100830006D655F746F5F6D61783A20000A00257501
:1008400000353A20776865656C5F6D61785F73701D
:100850006565643A20000A00257500343A20746901
:100860006D655F746F5F6D61783A20000A002575D1
:1008700000333A206D61785F73706565643A2000DB
:100880000A00257500323A20696E74657276616CD3
:10089000286D73293A20000A00257500313A20643A
:1008A000656C6179282A31306D73293A20000A0974
:1008B0002D2056616C756573202D0A004D3E004D4C
:1008C00025643E20003F0073657420646566617591
:1008D0006C740A00433E2000776865726520646589
:1008E0006C74613A20637572736F723D25642C20BD
:1008F000776865656C3D25640A5365652068747486
:10090000703A2F2F656E2E77696B69706564696127
:100910002E6F72672F77696B692F4D6F7573655FE7
:100920006B6579730A000A092D204D6F7573656B2D
:100930006579202D0A4553432F713A097175697401
:100940000A313A0964656C6179282A31306D73295E
:100950000A323A09696E74657276616C286D732982
:100960000A333A096D61785F73706565640A343AD9
:100970000974696D655F746F5F6D61780A353A0956
:10098000776865656C5F6D61785F73706565640A33
:10099000363A09776865656C5F74696D655F746F79
:1009A0005F6D61780A0A703A097072696E74207618
:1009B000616C7565730A643A0973657420646566D1
:1009C00061756C74730A75703A092B310A646F771C
:1009D0006E3A092D310A706775703A092B31300A69
:1009E0007067646F776E3A092D31300A0A7370654B
:1009F0006564203D2064656C7461202A206D6178F7
:100A00005F7370656564202A202872657065617463
:100A1000202F2074696D655F746F5F6D6178290A9E
:100A2000003F004D3E2000433E20004C25640A005C
:100A30000A092D20436F6E736F6C65202D0A455394
:100A4000432F713A09717569740A6D3A096D6F75B2
:100A500073656B65790A000A092D204D616769632A
:100A6000202D0A643A0964656275670A783A096458
:100A700065627567206D61747269780A6B3A096402
:100A800065627567206B6579626F6172640A6D3AA1
:100A9000096465627567206D6F7573650A763A093A
:100AA00076657273696F6E0A733A0973746174754F
:100AB000730A633A09636F6E736F6C65206D6F64C0
:100AC000650A302D343A096C61796572302D34280D
:100AD0004631302D4634290A506175733A09626FE8
:100AE0006F746C6F616465720A003F0074696D65B4
:100AF000725F72656164333228293A202530346C84
:100B0000580A006B6579626F6172645F69646C6535
:100B10003A2025580A006B6579626F6172645F70D4
:100B2000726F746F636F6C3A2025580A00686F7398
:100B3000745F6B6579626F6172645F6C6564732862
:100B4000293A2025580A000A092D2053746174752A
:100B500073202D0A004743433A20342E392E322089
:100B60004156522D4C4942433A20312E382E307393
:100B7000766E204156525F415243483A2061767268
:100B8000350A004F5054494F4E533A204C55464178
:100B9000204D4F5553454B45592045585452414BD4
:100BA000455920434F4E534F4C4520434F4D4D41E7
:100BB0004E44204B45594D41505F53454354494F96
:100BC0004E20343039360A004255494C443A2034DC
:100BD0003139303537312D646972747920283037D6
:100BE0003A35353A3537204F637420323820323069
:100BF0003137290A005649443A2030784645454461
:100C000028742E6D2E6B2E29205049443A203078BE
:100C1000343234322848484B42206D6F64292056C4
:100C200045523A203078303130340A00444553433D
:100C30003A20742E6D2E6B2E206B6579626F617277
:100C400064206669726D7761726520666F722048F4
:100C5000484B42206D6F640A000A092D20566572C8
:100C600073696F6E202D0A000A6D6F7573653A20E7
:100C70006F66660A000A6D6F7573653A206F6E0ABB
:100C8000000A6B6579626F6172643A206F66660A6A
:100C9000000A6B6579626F6172643A206F6E0A00B8
:100CA0000A6D61747269783A206F66660A000A6D8F
:100CB00061747269783A206F6E0A000A6465627521
:100CC000673A206F6E0A000A64656275673A206FA2
:100CD00066660A000A0A626F6F746C6F61646572FF
:100CE0002E2E2E2000433E20000011241FBECFEFE9
:100CF000DAE0DEBFCDBF04B603FE27C08091F70364
:100D00009091F803A091F903B091FA038730904BCA
:100D1000A740B04BD1F41092F7031092F803109251
:100D2000F9031092FA0314BE84B7877F84BF0FB60D
:100D3000F894A8958091600088618093600010927B
:100D400060000FBEE0E0F8E3099511E0A0E0B1E03B
:100D5000EEE5FCE502C005900D92AA39B107D9F77E
:100D600023E0AAE9B1E001C01D92A73FB207E1F775
:100D70000E944B100C942D2E0C9400000FB6809501
:100D80009AE0F8947BE27A95F1F708F0589A08F423
:100D9000589886959A95B1F70FBE08950FB680E8DA
:100DA000F894499BFECF4999FECF96E19A95F1F7C9
:100DB0009CE29A95F1F7869549998068C8F70FBE2D
:100DC00008950FB680E8F89496E19A95F1F79CE2C1
:100DD0009A95F1F7869549998068C8F796E19A95B2
:100DE000F1F7499BFECF0FBE0895FF93EF93E0917B
:100DF0009A01F0919B01309709F00995EF91FF91CD
:100E00000895FC018591803011F0EFDFFBCF08954C
:100E1000FF27E0E230E247FF0CC0419597FF09C091
:100E2000EDE26095709580959095611D711D811D15
:100E3000911D27FF02C0219530E350E2AA27660FDB
:100E4000771F881F991FAA1FA41710F0A41B639572
:100E50005A95A9F7AA3008F0A95FA05DAF93F39562
:100E6000611571058105910541F7ED3211F4EF939C
:100E7000F395F21718F43F93F395FBCF8F91B5DFFD
:100E8000FA95E1F70895E991F9918591803021F083
:100E9000853219F0AADFF9CF089520E0E894559142
:100EA0005532C1F3503311F4689455915A3348F4D4
:100EB000505390F3220F022E220F220F200D250FE8
:100EC000F4CF0EF4219589919991533619F3533744
:100ED00029F1533559F1BC0188279927E8945C36EC
:100EE00021F48991999168945591543639F446EFDB
:100EF0007EF077FF0DC08FEF9FEF0AC055374AE0B5
:100F000039F0583540E121F0523642E009F00895B9
:100F1000FF93EF937DDFEF91FF91B7CFFF93EF93B7
:100F2000FC0181918030B9F360DFFBCFFF93EF9339
:100F300068DFF1CFDF93CF93CDB7DEB72596A3DF80
:100F4000CF91DF91089514B88FEF85B9549A5C98CA
:100F500008958FEF84B980E485B9549A5C9A8FE143
:100F60009EE40197F1F700C0000008958FEF84B967
:100F700080E485B957985F9A87B1806C87B988B14A
:100F8000806C88B92E9A2F980E94A307ECEAF1E0B2
:100F900080E18E0F11928E13FDCFECE9F1E080E13C
:100FA0008E0F11928E13FDCF8CEA91E09093BF01CA
:100FB0008093BE018CE991E09093BD018093BC01C8
:100FC0000895EF92FF920F931F93CF93DF93809139
:100FD000BC019091BD012091BE013091BF013093C1
:100FE000BD012093BC019093BF018093BE015C9B27
:100FF0000E94A907C0E0D0E001E010E080E090E0AE
:10100000FC2FF770EC2FE87025B1207C2F2BAC0162
:1010100033E0440F551F3A95E1F7242B25B928B149
:101020002F73EE2311F0206401C0206828B92AE153
:101030002A95F1F700C0A091BC01B091BD01AC0FA1
:10104000BD1F2C9130E0082E02C0359527950A94DB
:10105000E2F720FD2F9AA5E3AA95F1F70000F6B478
:101060002E98BAE1BA95F1F700C04091BE015091B7
:10107000BF01BA016C0F7D1F4F9B0BC09801082E5A
:1010800001C0220F0A94EAF72095DB013C9123234B
:1010900009C0DB01EC909801082E01C0220F0A94D0
:1010A000EAF72E292C9326B56F2D70E02F1518F036
:1010B00026B530E004C026B530E021503F4F261B56
:1010C000370B2630310558F0A091BC01B091BD011D
:1010D000AC0FBD1F2C91DA01AC0FBD1F2C93BAE1F0
:1010E000BA95F1F700C02F982E9A20EA2A95F1F7C9
:1010F00001968830910509F087CFA091BE01B0918B
:10110000BF01AC0FBD1FE091BC01F091BD01EC0F20
:10111000FD1F9C918081981751F00E944425609397
:10112000C0017093C1018093C2019093C3012196C5
:10113000C031D10509F062CF5C9B1BC08091EE03EA
:10114000853021F08091EE03811113C06091C001C0
:101150007091C1018091C2019091C3010E947A25D2
:10116000613177428105910520F00E94A3070E941A
:10117000C52481E0DF91CF911F910F91FF90EF90F7
:1011800008952091BE013091BF01F901E80FF11DD2
:10119000808108950C94A9070C94A307569A81FFA7
:1011A00002C05E9A08955E98089588E08093CC000E
:1011B0001092CD00E9ECF0E080818069808380812D
:1011C00088608083EAECF0E080818083EBECF0E0E3
:1011D00080818083559A5D98789408959091C50197
:1011E0002091C4019217D1F030E0F901EA53FE4F8B
:1011F00080812F5F3F4F33272093C401492F50E058
:10120000921718F4241B350B03C0241B350B3395A0
:10121000233031050CF05D9890E008958FEF9FEF3B
:1012200008959091C80095FFFCCF8093CE0008955B
:101230001F920F920FB60F9211242F933F934F934B
:101240005F938F939F93EF93FF938091C50190E0FD
:10125000AC014F5F5F4F2091C401241741F03091E2
:10126000CE00FC01EA53FE4F30834093C50130911C
:10127000C501822F90E0432F50E0841B950B32175D
:1012800008F0939503970CF45D9AFF91EF919F916D
:101290008F915F914F913F912F910F900FBE0F90C3
:1012A0001F9018958091E002089508958091E002C2
:1012B00008950895089508950895CF93DF938D3C80
:1012C0009105B9F1B8F4853B9105A9F148F4833B48
:1012D0009105D1F1843B9105D1F5D0E0C0E23BC04E
:1012E000873B910571F150F18C3C910581F5D0E07F
:1012F000C8E031C08A3E9105C1F040F4823E9105BC
:10130000B1F0893E910519F5D0E124C0813222E087
:10131000920749F0833222E09207D9F08A3891404F
:10132000B1F4D2E017C0D4E015C0D0E213C0D0E4CD
:1013300011C0D0E80FC0D0E0C1E00DC0D0E0C2E0E5
:101340000AC0D0E0C4E007C0D0E0C0E104C0D0E0F3
:1013500001C0D1E0C0E08DEF0E94110983E00E943E
:10136000110983E00E9411098D2F0E9411098C2F11
:10137000DF91CF910C941109CF93DF93EC018DEFA6
:101380000E94110985E00E94110982E00E94110962
:1013900088810E94110989810E9411098A810E9415
:1013A00011098B81DF91CF910C941109CF93DF93B9
:1013B000EC018DEF0E94110989E00E94110981E082
:1013C0000E94110988810E94110980E00E94110980
:1013D0008A810E9411098B810E9411098C810E94CF
:1013E00011098D810E9411098E810E9411098F813E
:1013F000DF91CF910C9411090C94EE08EF92FF92BB
:101400000F931F93CF938C010E9438257C01C0E07D
:10141000C7010E9450258017910798F40E94EE089A
:101420009C012F3F8FEF380751F02D3041F02A30CB
:1014300041F0EC2FF0E0E853FD4F2083CF5FC73140
:1014400038F3EC2FF0E0E853FD4F108288EC92E087
:10145000CF911F910F91FF90EF9008950C94110977
:1014600081B3881F8827881F0895879A8F9A0895C7
:1014700085B7806885BF85B7806885BF0E94350ABB
:1014800086988E9A81988998559A5D980C94D5087B
:10149000879A8F9808958FB18695817008958FB13E
:1014A00086FB882780F908958093E0020895CF9302
:1014B000DF93FC018491EF012196882321F00E94A3
:1014C0001109FE01F7CFDF91CF910895CF93DF93FC
:1014D000C2EFD1E00E94EE088F3F2FEF920759F044
:1014E0009F938F93DF93CF930E949A070F900F9053
:1014F0000F900F90EFCFDF91CF9108950E94570A80
:101500002FEF89E698E1215080409040E1F700C03C
:10151000000084E690E00E94FE098093C60290934A
:10152000C7029F938F9385EF91E09F938F930E94C3
:101530009A070E94660A0F900F900F900F9080916B
:10154000C6029091C70208950E940D18909315014C
:10155000809314010E94011E80E091E00E9408180F
:101560000E94480A0E944F0A8111FCCF8DE792E049
:101570000E9401072FEF85EB95E3215080409040BA
:10158000E1F700C0000089E792E00E947E0AEFEFD9
:10159000FBE42DE1E150F0402040E1F700C0000005
:1015A0000E94660A85E792E00E947E0AFC01808123
:1015B000863721F081E792E00C947E0A089588E551
:1015C00092E00E94010782E592E00E947E0A0E945A
:1015D000350A0E94011E80911401909115010C940E
:1015E00008180C94870F8F929F92AF92BF92CF9260
:1015F000DF92EF92FF920F931F93CF93DF9392E0CE
:10160000B92E03EA14E029EAE22E24E0F22EAA24FD
:10161000A39433E0932E41E9C42E44E0D42E0E94DB
:10162000FC09EC01019609F441C08091E30281308C
:10163000F9F028F0823009F1833021F134C0CE3F37
:10164000D10519F4A092E302EACFC038D10528F4FD
:10165000DF93CF93FF92EF9204C0DF93CF931F935A
:101660000F930E949A070F900F900F900F90D7CF73
:101670002297C9F4B092E302D2CF2197A1F49092BD
:10168000E302CDCF8091D90380FF0AC0DF93CF93CF
:10169000DF92CF920E949A070F900F900F900F90B9
:1016A0008C2F0E94540A1092E302B9CF8091E50278
:1016B000811121C08091E40281111DC00E944B0A5A
:1016C00081110AC00E940D188A50914029F00E9491
:1016D000011E8AE091E00DC00E944B0A882359F058
:1016E0000E940D188651914031F00E94011E86E142
:1016F00091E00E9408188091E1029091E2020E941C
:101700005025893E23E0920708F461C028EE33E0BB
:10171000B9010E94DD2D629FC001639F900D729FF1
:10172000900D11242091E1023091E202820F931F6B
:101730009093E2028093E1020E942510833011F41D
:1017400081E001C080E00E94760F0E94442528EECF
:1017500033E040E050E00E94052E49015A018CE33D
:10176000C82ED12CE12CF12CCA01B901A701960198
:101770000E94052E672B682B692B49F50E94EE0FFE
:101780002091D90320FF23C09F938F931F921F9214
:10179000C501B40120E13EE040E050E00E94052E8A
:1017A000C22FA70196010E94052E3F932F931F92EF
:1017B000CF938CE794E09F938F930E949A078DB705
:1017C0009EB70A960FB6F8949EBF0FBE8DBF0E94BB
:1017D0004B0A811107C00E944F0A882319F06E9AA4
:1017E000769802C06E9A769ADF91CF911F910F91F1
:1017F000FF90EF90DF90CF90BF90AF909F908F9031
:1018000008958F929F92AF92BF92CF92DF92EF9204
:10181000FF921F93CF93DF9300D000D0CDB7DEB7F8
:10182000833109F48CC008F05BC08B3009F466C0CA
:101830008C3009F48FC0853009F0FBC10E9444252B
:1018400028EE33E040E050E00E94052E49015A01A5
:101850000E94EE0F9F938F938BEC92E09F938F9358
:101860000E949A07C501B40120E13EE040E050E04B
:101870000E94052E5F934F933F932F9325EC32E008
:101880003F932F9369837A838B839C830E949A076B
:101890008CE3C82ED12CE12CF12C69817A818B81CB
:1018A0009C81A70196010E94052E5F934F933F9361
:1018B0002F938FEB92E09F938F930E949A07C5011D
:1018C000B401A70196010E94052E9F938F937F93E9
:1018D0006F9389EB92E09F938F930E949A0740C188
:1018E000883361F020F4883109F440C1A2C1873403
:1018F00009F46DC18C3409F456C19BC188E594E0AC
:101900000E94010783E494E00E94010789E294E0C9
:101910000E94010782E094E00E94010787EE93E0B5
:101920000E94010785ED93E00E9401071091E502F6
:1019300011117DC185EB93E00E9401077EC10E94D9
:10194000A40A8DE992E00E947E0A87E992E00E9453
:101950007E0A6BC18CE993E00E9401070E940D187A
:101960008A50914019F08FE291E002C089E291E043
:101970009F938F938EE893E09F938F930E949A0793
:101980008091E4021F928F938FE793E09F938F9350
:101990000E949A070E944B0A0FB6F894DEBF0FBE52
:1019A000CDBF811107C00E944F0A811106C088E394
:1019B00091E005C084E391E002C08BE391E09F9346
:1019C0008F9385E793E09F938F930E949A070E94DD
:1019D000300A1F928F938AE593E09F938F930E9422
:1019E0009A078091E5021F928F9389E493E09F9379
:1019F0008F930E949A078091EE030FB6F894DEBF92
:101A00000FBECDBF8823B9F08091EE038130B1F0D5
:101A10008091EE038230A9F08091EE038330A1F033
:101A20008091EE03843099F08091EE03853091F03F
:101A300080E791E011C088E491E00EC080E491E07D
:101A40000BC083E591E008C08BE591E005C085E619
:101A500091E002C082E791E09F938F938AE393E045
:101A60009F938F930E949A0780E393E09F938F93B5
:101A70000E949A070E9425100F900F900F900F90D0
:101A80000F900F90813059F038F0823059F0833048
:101A900061F48AE193E00BC08BE293E008C085E239
:101AA00093E005C08EE193E002C088E193E09F934C
:101AB0008F930E949A070F900F9086E193E09F9377
:101AC0008F930E949A078091EC031F928F938DEF62
:101AD00092E09F938F930E949A078091D900817022
:101AE0001F928F9383EF92E09F938F930E949A07A8
:101AF0000E94442528EE33E040E050E00E94052E8D
:101B000069017A019CE3892E912CA12CB12CCA0188
:101B1000B901A50194010E94052E7F936F93C7011F
:101B2000B60120E13EE040E050E00E94052E122F79
:101B3000A50194010E94052E3F932F931F921F939E
:101B4000C701B60120E831E541E050E00E94052ED2
:101B50003F932F9386ED92E09F938F930E949A0775
:101B60000FB6F894DEBF0FBECDBF61C08091E50215
:101B7000811162C01091E402112339F08EEA92E0E3
:101B80000E9401071092E40258C084EA92E00E9489
:101B9000010781E08093E4020E94011E86E191E04A
:101BA0000E94081844C00E94300A182F882341F070
:101BB0000E94A40A81E08093E9038093E5023DC07E
:101BC0000E94DF0A1092E9031092E50230C0809172
:101BD000E502811102C00E94A40A8BE492E00E94F7
:101BE0007E0A80E492E00E947E0A8CE292E00E94EB
:101BF0007E0A85E292E00E947E0A8BE192E00E94DA
:101C00007E0A84E192E00E947E0A8AE092E00E94CD
:101C10007E0A80E092E00E947E0A8AEF91E00E94B4
:101C20007E0A8091E502811102C00E94DF0A11E064
:101C300004C01091E50201C010E0812F0F900F90B9
:101C40000F900F90DF91CF911F91FF90EF90DF9059
:101C5000CF90BF90AF909F908F900895CF93C82F53
:101C60000E94FA23827291E009F490E04C2F50E038
:101C7000FA013497E934F10508F0D0C0EA5AFF4F71
:101C80000C94272E8BE12DC19111CCC081E629C186
:101C90009111CAC082E625C19111C8C083E621C155
:101CA0009111C6C084E61DC19111C4C085E619C159
:101CB0009111C2C086E615C19111C0C087E611C15D
:101CC0009111BEC088E60DC19111BCC089E609C161
:101CD0009111BAC08AE605C19111B8C08BE601C165
:101CE0009111B6C08CE6FDC09111B4C08DE6F9C06B
:101CF0009111B2C08EE6F5C09111B0C08FE6F1C06F
:101D00009111AEC080E7EDC09111ACC081E7E9C090
:101D10009111AAC082E7E5C09111A8C083E7E1C094
:101D20009111A6C084E7DDC09111A4C085E7D9C098
:101D30009111A2C086E7D5C09111A0C087E7D1C09C
:101D400091119EC088E7CDC091119CC089E7C9C0A0
:101D500091119AC08AE7C5C0911198C081E3C1C0B2
:101D6000911196C082E3BDC0911194C083E3B9C0C4
:101D7000911192C084E3B5C0911190C085E3B1C0C8
:101D800091118EC086E3ADC091118CC087E3A9C0CC
:101D900091118AC088E3A5C0911188C089E3A1C0D0
:101DA000911186C080E39DC088E09BC089E099C006
:101DB00080E297C091117EC08DE293C091117CC0EA
:101DC0008DE38FC091117AC08BE58BC0911178C0E3
:101DD0008DE587C0992309F475C08CE782C09923EB
:101DE00009F472C08CE77DC0911170C08BE379C09B
:101DF00091116EC087E275C091116CC080E671C010
:101E000091116AC08CE26DC0911168C08EE269C008
:101E1000911166C08FE265C080E063C080E261C05E
:101E20008AE05FC081E45DC082E45BC083E459C0A6
:101E300084E457C085E455C086E453C087E451C0AC
:101E400088E44FC089E44DC08AE44BC08BE449C0AC
:101E50008CE447C08DE445C08EE443C08FE441C0AC
:101E600080E53FC081E53DC082E53BC083E539C0E8
:101E700084E537C085E535C086E533C087E531C0E8
:101E800088E52FC089E52DC08AE52BC081E229C0F5
:101E900080E427C083E225C084E223C085E221C01C
:101EA0008EE51FC086E21DC08AE21BC088E219C011
:101EB00089E217C08FE515C08BE213C08BE711C014
:101EC0008DE70FC08CE50DC08CE50BC08AE309C01F
:101ED00082E207C08EE705C08CE303C08EE301C039
:101EE0008FE30E942E0A81E0CF910895833019F488
:101EF000859A7D9A0895813011F4859A06C08230C2
:101F000019F4859A8D9A089585988D98089581E0A1
:101F10000E94760F2FEF81EE94E021508040904098
:101F2000E1F700C0000082E00E94760F2FEF81EE03
:101F300094E0215080409040E1F700C0000081E033
:101F40000E94760F2FEF81EE94E021508040904068
:101F5000E1F700C0000082E00E94760F2FEF81EED3
:101F600094E0215080409040E1F700C0000080E004
:101F70000E94760F80EC80937C0087E080937A004B
:101F800081E980937E0081E080937F008BE38093E2
:101F90007D00849A8C9808958091D90080FF1CC0A0
:101FA00090B331B385988D9AEFE9FFE03197F1F75F
:101FB00000C000008FB185FB882780F920B39072A4
:101FC0002F7D292B20BB91B3232F20729F7D922B35
:101FD00091BB91E08927089580E00895CF93DF9326
:101FE00000D0CDB7DEB7849A8C9A80917A00806851
:101FF00080937A008FE99FE00197F1F700C000001D
:1020000080917A00806480937A0080917A0086FDC6
:10201000FCCF80917800909179009A838983809198
:102020007A008F7780937A00849A8C9829813A81FC
:1020300045E0429FC001439F900D112480559109B6
:102040000F900F90DF91CF9108958091D90080FD7E
:102050000C94CC0F0E94EE0F8C3A2DE0920720F4E6
:1020600081E08093E60205C085379E4010F0109213
:10207000E6028091E602811102C082E0089583E0C9
:102080000895CF93C82F0E94BE068C2F0E94CE10B9
:1020900080E0CF91089584B7877F84BF0FB6F8940E
:1020A000A895809160008861809360001092600024
:1020B0000FBE90E080E80FB6F89480936100909393
:1020C00061000FBE0E9426150E9483158091E200D8
:1020D00084608093E20081E490E10E949624509A0B
:1020E000589A5198599A78948FEF9091EE038150B5
:1020F000943041F0EFE7FEE33197F1F700C00000C4
:102100008111F3CF8CEC94E00E9401070E94380A01
:102110000E94F10A80EC94E00E9401070E94CE1810
:102120000E944B0A811103C08AE091E002C086E15F
:1021300091E00E94081880EB94E00E9401070E9441
:102140004B0A882319F18091EE038530F9F48CEA6B
:1021500094E00E9401070E94CC080E94C5240E94BE
:10216000C5240E94C5240E94C5240E94C5240E9443
:10217000C5240E94C5248091EC03882301F30E94AA
:10218000EE248823E1F20E947B13D9CF0E94D2185B
:102190000E94F30AD4CF8091F30208959FB7F89478
:1021A0001092EA029FBF9091EE03943009F057C05D
:1021B0009091E9009F703091EC00232F217030FD49
:1021C00020E8922B24E02093E9002091EB0020FFEF
:1021D00043C02091EE0027FF3FC02091E702222359
:1021E00021F02091E80025FF37C01092E70226E099
:1021F0003091E80035FD15C03091EE03343061F5C3
:102200003091EB0035FD28C0215021F481E080930E
:10221000E70222C0EFE9FFE03197F1F700C00000CC
:10222000E7CF8093F1008091E80085FD0AC080919E
:10223000E80080FFFCCF8091E8008E778093E80073
:1022400006C08FB7F89421E02093EA028FBF9F70F9
:102250009093E90080E008959F709093E9008FEFDC
:102260000895CF93DF9300D01F92CDB7DEB79C01C6
:102270008091EE03843019F593E099833B832A83A0
:102280009093E9008FEF9091E800815095FD06C092
:1022900095ED9A95F1F700008111F5CF8091E80056
:1022A00085FF0DC040E050E063E070E0CE01019694
:1022B0000E9491138091E8008E778093E8000F9040
:1022C0000F900F90DF91CF910895CF93DF9300D0BF
:1022D0001F92CDB7DEB72091EE03243021F522E026
:1022E00029839B838A8383E08093E9008FEF909119
:1022F000E800815095FD06C095ED9A95F1F7000034
:102300008111F5CF8091E80085FF0DC040E050E0DD
:1023100063E070E0CE0101960E9491138091E80085
:102320008E778093E8000F900F900F90DF91CF9100
:1023300008952091EE032430F1F422E02093E90087
:102340002FEF3091E800215035FD06C035ED3A956C
:10235000F1F700002111F5CF2091E80025FF0BC017
:1023600040E050E065E070E00E9491138091E80049
:102370008E778093E8000895CF93DF932091EE034A
:10238000243039F521E02093E9002FEF3091E80067
:10239000215035FD06C035ED3A95F1F700002111C9
:1023A000F5CF2091E80025FF14C0EC0140E050E09B
:1023B00068E070E00E9491138091E8008E7780932E
:1023C000E80088E0FE01ABEEB2E001900D928A9544
:1023D000E1F7DF91CF9108958BED94E00E94010722
:1023E0008091ED03811109C00E9426150E9483157A
:1023F0008091E20084608093E200089587ED94E08C
:102400000E9401071092ED03089508952091E802BB
:102410002F5F822F62E30E94D12D992319F0209320
:10242000E80208951092E8028091EA02882371F18F
:102430008091EE03843041F58091E9008F70209106
:10244000EC00922F917020FD90E8892B94E09093FE
:10245000E9009091EB0090FF14C09091EE0097FF7F
:1024600010C09091E80095FF03C01092F100F9CFE1
:102470009091E80090FF05C09091E8009E779093BE
:10248000E8008F708093E9001092EA02089542E01C
:1024900061EC81E00E94A01442E061EC82E00E94C5
:1024A000A01442E061EC83E00E94A01442E261ECDF
:1024B00084E00C94A0148091F003833009F453C09D
:1024C00030F4813071F0823009F48CC008958A3084
:1024D00009F478C08B3009F45EC0893009F09AC0E5
:1024E00020C08091EF03813A09F094C08091E80008
:1024F000877F8093E8008091F3039091F403892B08
:1025000021F468E08BEE92E003C060E080E090E0B0
:1025100070E00E94DC138091E8008B778093E800E4
:1025200008958091EF03813209F074C08091F30324
:102530009091F403892B09F06DC08091E800877FAA
:102540008093E8008091E80082FD05C08091EE0351
:102550008111F8CF5FC08091F1008093F3028091E8
:10256000E8008B7753C08091EF03813A09F052C0A5
:102570008091F3039091F403892B09F04BC0809173
:10258000E800877F8093E8008091E80080FFFCCF1F
:102590008091200136C08091EF038132D9F580917E
:1025A000F3039091F403892BA9F58091E800877FCC
:1025B0008093E8000E94D5148091F103809320015C
:1025C0000C94011E8091EF03813221F58091E80087
:1025D000877F8093E8000E94D5148091F203809356
:1025E000F40208958091EF03813AA1F48091E8000C
:1025F000877F8093E8008091E80080FFFCCF809186
:10260000F4028093F1008091E8008E778093E800D7
:102610000C94D51408958091F3028093E9021092EE
:10262000F30280E00E94CE080E949F190C94011EC4
:102630000C940B130E9402258091E9028093F3020F
:1026400008950C941A13292F332723303105C9F02C
:1026500064F42130310581F02230310509F043C0A6
:1026600084E790E027E035E042C021323105F1F007
:102670002232310541F137C082E190E02BE735E0AD
:1026800036C099278130910541F08230910541F0A3
:10269000892B49F5E3E0F5E005C0E3EFF4E002C083
:1026A000EFEDF4E0849190E09F0121C06430D8F414
:1026B000E62FF0E0EE0FFF1FE857FE4F208131813B
:1026C00089E090E014C0643070F470E0FB01EE0F1C
:1026D000FF1FE058FE4F20813181FB01E458FE4F7F
:1026E000808190E004C080E090E020E030E0FA01DA
:1026F00031832083089580E189BD82E189BD09B4D9
:1027000000FEFDCF8091D8008F7D8093D80080910E
:10271000E00082608093E0008091E00081FDFCCFCA
:102720000895CF92DF92EF92FF920F931F93CF9372
:10273000DF93EC018B016A010E94F414811133C014
:10274000C114D10439F0F60180819181081B190B65
:10275000C80FD91FE12CF12C0115110519F1809139
:10276000E80085FD16C08091E8008E778093E80030
:10277000C114D10449F0F60180819181E80EF91E5F
:10278000F182E08285E00FC00E94F414882321F3D7
:102790000AC089918093F10001501109FFEFEF1AEF
:1027A000FF0ADACF80E0DF91CF911F910F91FF9068
:1027B000EF90DF90CF9008952091F5033091F603CC
:1027C0002617370748F06115710539F42091E800A4
:1027D0002E772093E80001C0B90140E06115710532
:1027E000A9F12091EE03222309F443C0253009F416
:1027F00042C02091E80023FD40C02091E80022FD66
:1028000032C02091E80020FFE9CF4091F3002091F1
:10281000F20030E0342BFC01CF016115710559F055
:102820002830310540F481918093F10061507109A5
:102830002F5F3F4FF1CF41E02830310509F040E0F4
:102840002091E8002E772093E800C8CF4111C9CF2E
:102850000AC08091EE03882361F0853061F0809199
:10286000E80083FD0AC08091E80082FFF2CF80E09B
:10287000089582E0089583E0089581E0089520910D
:10288000F5033091F6032617370748F061157105F7
:1028900039F42091E8002E772093E80001C0B901B7
:1028A000FC0120E06115710591F18091EE03882310
:1028B00009F440C0853009F43FC08091E80083FDF1
:1028C0003DC08091E80082FD2FC08091E80080FF2C
:1028D000E9CF2091F3008091F20090E0922B6115F6
:1028E000710559F08830910540F424912093F1004E
:1028F0003196615071090196F2CF21E0089709F0F5
:1029000020E08091E8008E778093E800CBCF211102
:10291000CCCF0AC08091EE03882361F0853061F04E
:102920008091E80083FD0AC08091E80082FFF2CF29
:1029300080E0089582E0089583E0089581E008959D
:10294000982F973058F59093E900981739F07091C7
:10295000EC002091ED005091F00003C0242F762F61
:1029600050E021FF19C03091EB003E7F3093EB0027
:102970003091ED003D7F3093ED003091EB00316000
:102980003093EB007093EC002093ED005093F00037
:102990002091EE0027FF07C09F5FD3CF8F708093F9
:1029A000E90081E0089580E008958091EF0387FFBA
:1029B00011C08091E80082FD05C08091EE03811175
:1029C000F8CF11C08091E8008B770BC08091EE03A7
:1029D000882349F08091E80080FFF8CF8091E800DB
:1029E0008E778093E80008952091E4003091E5000F
:1029F00095E64091EC00842F817040FF22C08091C9
:102A0000E80080FD1CC08091EE03882391F08530A2
:102A100091F08091EB0085FD10C04091E400509151
:102A2000E5004217530729F39A01915011F784E00A
:102A3000089582E0089583E0089581E0089580E09C
:102A400008954091E80042FFDECF08950E9494155A
:102A50000E949C15E0EEF0E0808181608083E8EDCB
:102A6000F0E080818F77808319BCA7EDB0E08C9176
:102A70008E7F8C9380818F7E80831092ED030895EA
:102A80000F931F93CF93DF930E9494150E949C1580
:102A9000C8EDD0E088818F778883888180688883BB
:102AA00088818F7D888319BC1092EE031092EA030F
:102AB0001092EC031092EB0300EE10E0F80180811D
:102AC0008B7F808388818160888342E060E080E042
:102AD0000E94A014E1EEF0E080818E7F8083E2EE20
:102AE000F0E0808181608083808188608083F8014C
:102AF00080818E7F8083888180618883DF91CF9100
:102B00001F910F910895E8EDF0E080818F7E808322
:102B1000E7EDF0E080818160808384E082BF81E026
:102B20008093ED030C944015E8EDF0E080818E7FFA
:102B300080831092E20008951092DA001092E10072
:102B400008951F920F920FB60F9211242F933F9367
:102B50004F935F936F937F938F939F93AF93BF93A5
:102B6000EF93FF938091E10082FF0BC08091E20020
:102B700082FF07C08091E1008B7F8093E1000E947B
:102B800006128091DA0080FF1FC08091D80080FF7C
:102B90001BC08091DA008E7F8093DA008091D9008B
:102BA00080FF0DC080E189BD82E189BD09B400FECE
:102BB000FDCF81E08093EE030E94EC1105C019BCAB
:102BC0001092EE030E94FE118091E10080FF19C077
:102BD0008091E20080FF15C08091E2008E7F80939B
:102BE000E2008091E20080618093E2008091D80051
:102BF00080628093D80019BC85E08093EE030E9428
:102C000018138091E10084FF30C08091E20084FFBE
:102C10002CC080E189BD82E189BD09B400FEFDCFF1
:102C20008091D8008F7D8093D8008091E1008F7EC5
:102C30008093E1008091E2008F7E8093E20080919A
:102C4000E20081608093E2008091EA03882311F022
:102C500084E007C08091E30087FD02C081E001C0ED
:102C600083E08093EE030E9421138091E10083FFB3
:102C700029C08091E20083FF25C08091E100877F19
:102C80008093E10082E08093EE031092EA0380914A
:102C9000E1008E7F8093E1008091E2008E7F80933F
:102CA000E2008091E20080618093E20042E060E017
:102CB00080E00E94A0148091F00088608093F00072
:102CC0000E940512FF91EF91BF91AF919F918F915B
:102CD0007F916F915F914F913F912F910F900FBE18
:102CE0000F901F9018951F920F920FB60F921124FC
:102CF0002F933F934F935F936F937F938F939F9304
:102D0000AF93BF93CF93DF93EF93FF93C091E9000D
:102D1000CF708091EC00D82FD17080FDD0E8109258
:102D2000E9008091F000877F8093F00078940E9402
:102D3000B7161092E9008091F00088608093F0004F
:102D4000CD2BCF70C093E900FF91EF91DF91CF9130
:102D5000BF91AF919F918F917F916F915F914F91B3
:102D60003F912F910F900FBE0F901F9018951F93BA
:102D7000CF93DF93CDB7DEB7AA970FB6F894DEBF37
:102D80000FBECDBFEFEEF3E088E08E0F9091F10023
:102D900091938E13FBCF0E945B128091E80083FF1A
:102DA0001FC18091EF039091F003492F50E04A300A
:102DB000510508F015C1FA01E156FF4F0C94272E7A
:102DC000803881F0823809F00BC18091F3038F7055
:102DD0008093E9008091EB0085FB882780F91092B1
:102DE000E90006C08091EB039091EC0391118260A1
:102DF0009091E800977F9093E8008093F100109203
:102E0000F100C8C0282F2D7F09F0EAC0882319F0EF
:102E1000823061F0E5C08091F103813009F0E0C0BB
:102E2000933009F080E08093EC032BC08091F10394
:102E3000811127C08091F3038F7009F4D1C0809372
:102E4000E9002091EB0020FF1CC0933021F4809119
:102E5000EB00806214C09091EB0090619093EB00C6
:102E600021E030E0A90102C0440F551F8A95E2F726
:102E70004093EA001092EA008091EB008860809312
:102E8000EB001092E9008091E800877F86C08111F5
:102E9000A7C01091F1031F778091E3008078812B08
:102EA0008093E3008091E800877F8093E8000E9490
:102EB000D5148091E80080FFFCCF8091E30080680A
:102EC0008093E300111102C082E001C083E080938F
:102ED000EE0386C08058823008F082C08091F103F2
:102EE0009091F2038C3D53E0950779F583E08A8356
:102EF0008AE289834FB7F894DE01139620E03EE022
:102F000051E2E32FF0E050935700E49120FF03C01B
:102F1000E295EF703F5FEF708E2F90E0EA3010F097
:102F2000C79601C0C0968D939D932F5F243149F7BA
:102F30004FBF8091E800877F8093E8006AE270E0ED
:102F4000CE0101960E94DC1314C0AE014F5F5F4FAB
:102F50006091F3030E942313BC01892B09F440C044
:102F60009091E800977F9093E80089819A810E9470
:102F70003F148091E8008B778093E80031C080385F
:102F800079F58091E800877F8093E8008091EA03DB
:102F90008093F1008091E8008E778093E8000E9492
:102FA000D5141EC081111CC09091F1039230C0F461
:102FB0008091E800877F8093E8009093EA030E9465
:102FC000D5148091EA03811106C08091E30087FD4A
:102FD00002C081E001C084E08093EE030E944712AA
:102FE0008091E80083FF0AC08091E800877F80938A
:102FF000E8008091EB0080628093EB00AA960FB608
:10300000F894DEBF0FBECDBFDF91CF911F91089521
:103010009093FA028093F90208958091F9029091B9
:10302000FA020895E091F902F091FA02309721F046
:103030000190F081E02D099480E00895EF92FF92D5
:103040000F931F93CF93DF93E091F902F091FA026F
:103050003097B1F18C010280F381E02D09958091C8
:10306000D90382FF2DC080FF04C088E996E00E944A
:103070000107E80118E082E9E82E86E0F82E809149
:10308000D90380FF0BC088811F928F93FF92EF922C
:103090000E949A070F900F900F900F901150219659
:1030A0001111EDCF8091D90380FF0AC080E996E02D
:1030B000DF91CF911F910F91FF90EF900C9401073A
:1030C000DF91CF911F910F91FF90EF900895E091C4
:1030D000F902F091FA02309721F00480F581E02D99
:1030E00009940895CF93DF93EC018091F7029091BA
:1030F000F802C817D90709F1D093F802C093F70274
:10310000E091F902F091FA023097B9F00680F78168
:10311000E02DCE0109958091D90382FF0EC080FF7A
:103120000CC0DF93CF9382E896E09F938F930E9429
:103130009A070F900F900F900F90DF91CF91089505
:10314000CF93DF93EC018091F5029091F602C817BE
:10315000D90709F1D093F602C093F502E091F90284
:10316000F091FA023097B9F00084F185E02DCE019C
:1031700009958091D90382FF0EC080FF0CC0DF93B8
:10318000CF9382E796E09F938F930E949A070F90C8
:103190000F900F900F90DF91CF9108950E942F25EF
:1031A0000C94B6075F926F927F928F929F92AF922C
:1031B000BF92CF92DF92EF92FF920F931F93CF9324
:1031C000DF9300D000D01F92CDB7DEB70E94E10799
:1031D0008CEFC82E82E0D82E512C88248394912C19
:1031E000852D0E94C108A82EF601E080E82641F452
:1031F0005394FFEFCF1ADF0A80E15812F1CF40C09D
:103200008091D90381FD0E94A01900E010E0F12C0B
:10321000B12CC701002E02C0959587950A94E2F75C
:1032200080FF28C009835A823401002E02C0660C38
:10323000771C0A94E2F793012A213B2181E0232B9A
:1032400009F480E08B830E9438258160782F9D836C
:103250008C8349815A816B818D810E94D419498167
:103260005A816B817C818D810E94B224F60180811C
:10327000682660820F5F1F4F0830110551F6B8CFE6
:103280008FEF89838A831B820E9438258160782F83
:103290009D838C8349815A816B818D810E94D419D1
:1032A0000E94B1240E9425281091FB020E9412184E
:1032B000181771F10E9412188093FB029091D903A4
:1032C00092FF0EC090FF0CC01F928F9383EA96E08E
:1032D0009F938F930E949A070F900F900F900F90DB
:1032E0008091FB020F900F900F900F900F90DF9145
:1032F000CF911F910F91FF90EF90DF90CF90BF90F3
:10330000AF909F908F907F906F905F900C94C324AC
:103310000F900F900F900F900F90DF91CF911F9112
:103320000F91FF90EF90DF90CF90BF90AF909F9064
:103330008F907F906F905F9008950C94CE080895C1
:10334000EF92FF920F931F93CF93DF938CEB96E056
:103350000E940107C0E0D0E08EE2E82E81E0F82E66
:103360000EEA16E08C2F0E94C1080E949B24FF9257
:10337000EF921F928F93DF93CF931F930F930E942F
:103380009A0721968DB79EB708960FB6F8949EBF00
:103390000FBE8DBFC031D10529F7DF91CF911F91AD
:1033A0000F91FF90EF900895CF93DF93CDB7DEB7E5
:1033B0002B970FB6F894DEBF0FBECDBF942F4F836F
:1033C000252F588769877A878B874A855B85452BA8
:1033D00021F02F3F09F59F3FF9F4DE01119686E0B9
:1033E000FD0111928A95E9F785E0FE01379601907B
:1033F0000D928A95E1F749815A816B817C818D819B
:103400009E810E94E6202B960FB6F894DEBF0FBE79
:10341000CDBFDF91CF9108954F81588569857A8519
:103420008B850E94B224D9CFCF93882309F465C03D
:10343000C82F8CEF8C0F813A20F080E58C0F8E32F4
:1034400048F48C2F0E944B2B811157C08C2F0E9467
:10345000BE230CC080E28C0F883058F4C77081E026
:1034600001C0880FCA95EAF70E94FD23CF910C9402
:1034700041248BE58C0F833078F4C53A29F0C63AA5
:1034800031F083E890E005C081E890E002C082E876
:1034900090E0CF910C94721888E58C0F853168F517
:1034A000C83A89F0C93A91F0CA3A99F0CB3AA1F0FA
:1034B000CC3AA9F0CD3AB1F0CE3AB9F0CF3AC1F05A
:1034C00080E090E017C082EE90E014C089EE90E0BA
:1034D00011C08AEE90E00EC085EB90E00BC086EB49
:1034E00090E008C083EB90E005C084EB90E002C060
:1034F00087EB90E0CF910C94A018CF91089588238A
:1035000049F19CEF980F913A20F090E5980F9E3288
:1035100018F40E94DB230DC090E2980F983058F405
:10352000877091E001C0990F8A95EAF7892F0E9470
:1035300003240C9441249BE5980F933020F480E001
:1035400090E00C947218885A853120F480E090E065
:103550000C94A0180895882321F00E94FD230C9458
:1035600041240895882321F00E9403240C944124CF
:103570000895BF92CF92DF92EF92FF920F931F9325
:10358000CF93DF9300D000D000D0CDB7DEB725E0D9
:10359000FC01DE01119601900D922A95E1F7FC01E4
:1035A00040815181028163817481258122952F7030
:1035B0006115710509F403C35F3F19F44F3F09F426
:1035C000FEC26C01862F7D836C83602F782F8D81E6
:1035D0002E830E944223182FB92E0E9441230E945D
:1035E0003122EB2DE295EF70F0E0E755FF4F2E8191
:1035F0000C94272E8B2D807F9B2D9F70F92E882376
:1036000019F0F29490EFF922002349F0FF2009F419
:1036100083C28F2D0E9410240E9441247DC2812FDD
:103620000E947F1AFF2009F4CAC28F2D0E9416241F
:1036300026960FB6F894DEBF0FBECDBFDF91CF91B7
:103640001F910F91FF90EF90DF90CF90BF900C945F
:1036500041248B2D807F9B2D9F70F92E803219F095
:10366000F29480EFF822112319F0113009F12AC0E9
:103670000023B1F08F2D222351F1213041F5269600
:103680000FB6F894DEBF0FBECDBFDF91CF911F9173
:103690000F91FF90EF90DF90CF90BF900C9420247B
:1036A000222319F0213009F48AC20E9429242DC056
:1036B0000023F1F0263008F082C20E94FA238F2105
:1036C00029F023C00023F9F0211116C08F2D269672
:1036D0000FB6F894DEBF0FBECDBFDF91CF911F9123
:1036E0000F91FF90EF90DF90CF90BF900C94AB1AAA
:1036F000253008F064C209C0F601858180FF0CC244
:103700008F708583E3CF21111CC28F2D83C12B2D98
:1037100026952695237030E02115310521F02130C2
:103720003105D1F04CC2002321F0812F9B2D9370E5
:1037300002C080E090E026960FB6F894DEBF0FBE80
:10374000CDBFDF91CF911F910F91FF90EF90DF9050
:10375000CF90BF900C947218002321F0812F9B2DE5
:10376000937002C080E090E026960FB6F894DEBF1A
:103770000FBECDBFDF91CF911F910F91FF90EF90C2
:10378000DF90CF90BF900C94A018812F002319F0E8
:103790000E94AB2602C00E94132726960FB6F8940B
:1037A000DEBF0FBECDBFDF91CF911F910F91FF9074
:1037B000EF90DF90CF90BF900C9498278B2D837063
:1037C00009F07BC00111FBC1812F8295869587701E
:1037D000880F880F912F9F70C92ED12CE12CF12CCE
:1037E000082E04C0CC0CDD1CEE1CFF1C0A94D2F782
:1037F00014FF12C04FE050E060E070E004C0440FDE
:10380000551F661F771F8A95D2F7CB01BA016095C5
:1038100070958095909503C060E070E0CB012B2DF2
:10382000269526952370422F50E042305105D9F05D
:103830004330510569F16C297D298E299F2941303A
:10384000510551F126960FB6F894DEBF0FBECDBFDD
:10385000DF91CF911F910F91FF90EF90DF90CF906C
:10386000BF900C9456226C297D298E299F2926967B
:103870000FB6F894DEBF0FBECDBFDF91CF911F9181
:103880000F91FF90EF90DF90CF90BF900C9470223B
:103890000E945622C701B60126960FB6F894DEBFE5
:1038A0000FBECDBFDF91CF911F910F91FF90EF9091
:1038B000DF90CF90BF900C943C22002319F08B2D09
:1038C000817001C08695882309F479C1812F829582
:1038D00086958770880F880F912F9F70C92ED12CE5
:1038E000E12CF12C082E04C0CC0CDD1CEE1CFF1CBE
:1038F0000A94D2F714FF12C04FE050E060E070E08D
:1039000004C0440F551F661F771F8A95D2F7CB015D
:10391000BA01609570958095909503C060E070E065
:10392000CB012B2D269526952370422F50E0423057
:103930005105D9F04330510569F16C297D298E2953
:103940009F294130510551F126960FB6F894DEBFFC
:103950000FBECDBFDF91CF911F910F91FF90EF90E0
:10396000DF90CF90BF900C941D236C297D298E2968
:103970009F2926960FB6F894DEBF0FBECDBFDF910C
:10398000CF911F910F91FF90EF90DF90CF90BF905C
:103990000C942F230E941D23C701B60126960FB653
:1039A000F894DEBF0FBECDBFDF91CF911F910F9175
:1039B000FF90EF90DF90CF90BF900C940B23103FBF
:1039C000D1F128F480E4810F803250F0A0C0123F82
:1039D00009F462C008F44BC0133F09F472C097C0E9
:1039E000F12FF071FF2E8B2D8F71002351F00E946B
:1039F000A422812FFF2019F08295807F68CE8F70DE
:103A000066CE0E94C522812FFF2019F08295807F0B
:103A100001C08F7026960FB6F894DEBF0FBECDBFE3
:103A2000DF91CF911F910F91FF90EF90DF90CF909A
:103A3000BF900C94B21A0023B1F0253008F0BFC03B
:103A40008B2D8F7126960FB6F894DEBF0FBECDBFBB
:103A5000DF91CF911F910F91FF90EF90DF90CF906A
:103A6000BF900C94EA22263008F0A9C0E9CF0023C9
:103A7000A9F08B2D8F7126960FB6F894DEBF0FBE7E
:103A8000CDBFDF91CF911F910F91FF90EF90DF900D
:103A9000CF90BF900C94A422002359F38B2D8F71EB
:103AA00026960FB6F894DEBF0FBECDBFDF91CF9143
:103AB0001F910F91FF90EF90DF90CF90BF900C94EB
:103AC000C522002399F08B2D8F7126960FB6F8949E
:103AD000DEBF0FBECDBFDF91CF911F910F91FF9041
:103AE000EF90DF90CF90BF900C948F2226960FB668
:103AF000F894DEBF0FBECDBFDF91CF911F910F9124
:103B0000FF90EF90DF90CF90BF900C948A2200231B
:103B1000A9F0222309F4ADCF812F26960FB6F89491
:103B2000DEBF0FBECDBFDF91CF911F910F91FF90F0
:103B3000EF90DF90CF90BF900C94141A222309F4D9
:103B4000ADCF812F26960FB6F894DEBF0FBECDBF46
:103B5000DF91CF911F910F91FF90EF90DF90CF9069
:103B6000BF900C947F1A4B2D4F70612FC6010E949D
:103B7000252626960FB6F894DEBF0FBECDBFDF9187
:103B8000CF911F910F91FF90EF90DF90CF90BF905A
:103B90000C948A214B2D4F70612FC60126960FB6CB
:103BA000F894DEBF0FBECDBFDF91CF911F910F9173
:103BB000FF90EF90DF90CF90BF900C942826269630
:103BC0000FB6F894DEBF0FBECDBFDF91CF911F912E
:103BD0000F91FF90EF90DF90CF90BF9008950E94DB
:103BE0001D240E94EC230E9441240E94CA280E94A6
:103BF000982780E090E00E94721880E090E00C949A
:103C0000A0180E940D240C94EF1DCF93DF9300D0D9
:103C100000D01F92CDB7DEB7942F4983252F5A834A
:103C20006B837C838D834C815D81452B39F12F3FE4
:103C300011F49F3F19F149815A816B817C818D81FB
:103C40000E944223292F22952F7030E02C3031051D
:103C500004F52A3031055CF4225031092230310557
:103C600068F4853A80F4843090F4823080F0883EA5
:103C700038F4803E60F48450813A48F080E014C00B
:103C8000803FE1F704C090E2980F983080F781E020
:103C90000BC02C30310521F493FB882780F904C038
:103CA0002F303105C9F3EACF0F900F900F900F908E
:103CB0000F90DF91CF910895CF93DF9300D000D084
:103CC0001F92CDB7DEB70F900F900F900F900F900F
:103CD000DF91CF910895CF93DF9300D000D000D033
:103CE000CDB7DEB726960FB6F894DEBF0FBECDBFB8
:103CF000DF91CF9108951F93CF93DF93C0910C0371
:103D000016E080910D03C81799F0D0E01C9FF001D8
:103D10001D9FF00D1124E25FFC4F408151816281B3
:103D20007381848195810E946B1E2196C770E9CFB3
:103D3000DF91CF911F91089540913E0350913F0331
:103D4000609140037091410380914203909143033D
:103D50000C946B1E8091430382958F7009F054C0C0
:103D600080914003882309F44FC080910C03A091F7
:103D70000D0360913E0370913F03409141035091C8
:103D80004203B6E08A1709F43FC090E0411551059F
:103D9000C1F17F3F11F46F3FA1F1B89FF001B99FCE
:103DA000F00D1124E25FFC4F218172132AC02081A3
:103DB000621327C02281211124C02381348124175A
:103DC000350710F421503109241B350B2C323140BA
:103DD000C0F4209143032F7020612093430326E019
:103DE000289FF001299FF00D1124ED5EFC4F80818A
:103DF0008F70806180838EE393E00E94B91A0C94E7
:103E00007B1E01968770BECF0895BF92CF92DF923E
:103E1000EF92FF920F931F93CF93DF93CDB7DEB74F
:103E200061970FB6F894DEBF0FBECDBF7C0185E071
:103E3000F701DE011D9601900D928A95E1F7D701F9
:103E40004C9111965C9111971296DC9012971396F3
:103E50000D911C91149730913E0360913F03809126
:103E6000410390914203009709F47FC16F3F19F419
:103E70003F3F09F47AC1B0904003BB2009F4CAC0A7
:103E8000209143030817190750F0F801E81BF90BBC
:103E9000CF01CC24C3948C329140D0F009C08095DE
:103EA0009095800F911FCC24C3948C32914080F068
:103EB000C12C207F09F0CCC0702F198B088B6D2D81
:103EC00089890E945C1E8EE393E00E94B91AB6C0F5
:103ED000822F807F09F047C0651314C0341312C0CD
:103EE000D11010C02F702061209343030E949C1EAC
:103EF0008EE393E00E94B91A80914303D70115968F
:103F00008C932FC00115110519F15F3F11F44F3F3C
:103F1000F9F0CD2CD1101CC080910C0320910D0321
:103F200036E0821709F45CC090E0389FF001399FB9
:103F3000F00D1124E25FFC4F6181561306C06081D1
:103F4000461303C06281611103C001968770E9CFF7
:103F5000CD2CDD2009F429C1809143038160809339
:103F60004303C12C22C1651308C0341306C0D1100D
:103F700004C080914303D701CCC04D875E87DF86A4
:103F8000702F198B088B6D2D89890E94051E88233F
:103F9000E9F1DD20D9F120914303822F82958F70C2
:103FA00090E0029774F080913E0390913F039887D0
:103FB0008F8319861B870A872C87CE0107960E945C
:103FC000B91A86E0F701AEE3B3E001900D928A954D
:103FD000E1F70E94AA1E0E949C1ECC24C394E5C057
:103FE000702F198B088B60E089890E944223292F4A
:103FF00022952F7030E0223031050CF0CAC09F703E
:1040000009F0C4C0805E883008F4CFC0C7010E94A8
:10401000B91AE3CF0817190708F456C0F801E81BCE
:10402000F90BCF018C32914008F456C0C12C702F8F
:10403000198B088B6D2D89890E945C1EEEE3F3E0DD
:1040400086E0DF011D928A95E9F70E949C1EADC0B3
:10405000651314C0341312C0D11010C080914303F3
:10406000F7018583C7010E94B91A86E0EEE3F3E009
:10407000DF011D928A95E9F7CB2C97C04D875E87AB
:10408000DF86702F198B088B6D2D89890E94051E84
:10409000882309F4BBCFDD2009F4B8CF2091430376
:1040A000822F82958F7090E002970CF48ACF8091D6
:1040B0003E0390913F039A8389831B821D830C8367
:1040C0002E83CE0101967BCF80959095800F911F16
:1040D0008C32914008F0AACFCD2CDD2009F496CF88
:1040E00065132EC034132CC02091430320FD1FC044
:1040F000822F82958F70D9F0D70115962C93159742
:104100008F3049F08F5F982F9295907F822F8F701C
:10411000892B15968C93C7010E94B91A86E0F70186
:10412000AEE3B3E001900D928A95E1F78ECF86E081
:10413000F701AEE3B3E001900D928A95E1F735C047
:104140004D875E87DF86702F198B088B6D2D8989CF
:104150000E94051E811135CF8091430381608093B9
:104160004303C7010E94B91A20C0DD2009F44ECFD5
:104170004D875E87DF86702F198B088B6D2D89899F
:104180000E94051E882309F441CF1BCF81113ACF2D
:104190000CC0243031050CF039CF9F7009F432CFB8
:1041A000F7019581907F09F02DCF8C2D61960FB688
:1041B000F894DEBF0FBECDBFDF91CF911F910F915D
:1041C000FF90EF90DF90CF90BF9008951F93CF9313
:1041D000DF93CDB7DEB72C970FB6F894DEBF0FBED6
:1041E000CDBF4F83588769877A878B879C87CE019D
:1041F00007960E94051F882369F08F8198852A857C
:104200003B85232BF1F19F3F09F063C08F3F09F0FD
:1042100060C037C086E0FE013796DE01119601903E
:104220000D928A95E1F76F817885EA85FB85309755
:1042300041F17F3F11F46F3F21F120910D0330E0F8
:10424000C90101968770992740910C0350E08417AB
:10425000950709F447C069837A83FD83EC8396E070
:10426000929FD001939FB00D1124A25FBC4FFE011D
:10427000319601900D929A95E1F780930D030E947B
:104280007B1E16E080910C0390910D038917C1F1FC
:10429000189FC0011124825F9C4F0E94051F882334
:1042A00079F1E0910C031E9FF0011124E25FFC4FB5
:1042B0004081518162817381848195810E946B1E4E
:1042C00080910C0390E001968770992780930C03EE
:1042D000D9CF4F81588569857A858B859C850E94C9
:1042E0006B1ECFCF0E94011E10920D0310920C0383
:1042F000EEE3F3E086E0DF011D928A95E9F7C1CF96
:104300002C960FB6F894DEBF0FBECDBFDF91CF91D4
:104310001F910895DF92EF92FF920F931F93CF9317
:10432000DF93FC01892B09F48AC0E12CF12CDD24F8
:10433000D394EF0121968491853709F461C058F434
:10434000843708F04EC0843008F06AC08130D1F064
:10435000823071F174C0883709F45DC050F486373B
:1043600009F455C0873709F06AC08E2D0E940A24CF
:1043700054C09CE7980F903708F061C08F770E9477
:104380007F1A50C08F010E5F1F4FFE01849190E293
:10439000980F983050F48770FD2D01C0FF0F8A955B
:1043A000EAF78F2F0E94102414C00E94141A13C021
:1043B0008F010E5F1F4FFE01C49180E28C0F883089
:1043C00060F4C7708D2D01C0880FCA95EAF70E946E
:1043D00016240E944124E80125C08C2F0E947F1AD8
:1043E000FACF9F012E5F3F4FFE01C491CC2369F0AD
:1043F0008FE99FE00197F1F700C00000C150F6CFB0
:104400009F012E5F3F4FFE01F490E9010BC00E9417
:10441000FA23E82E07C00E940D240E94412402C006
:104420000E94141A8F2D882341F0EFE9FFE03197A5
:10443000F1F700C000008150F6CFFE017ACFDF9186
:10444000CF911F910F91FF90EF90DF9008956093AF
:10445000C4037093C5038093C6039093C7030C9461
:10446000C22408956093C8037093C9038093CA035C
:104470009093CB030C94C1240F931F930091C80316
:104480001091C9032091CA033091CB03602B712B8B
:10449000822B932B6093C8037093C9038093CA0344
:1044A0009093CB031F910F910C94C1240F931F93F2
:1044B0000091C8031091C9032091CA033091CB0326
:1044C00060237123822393236093C8037093C903ED
:1044D0008093CA039093CB031F910F910C94C12436
:1044E0000F931F930091C8031091C9032091CA0331
:1044F0003091CB0360277127822793276093C803ED
:104500007093C9038093CA039093CB031F910F91BB
:104510000C94C12460E070E0CB010C9427220F932F
:104520001F9341E050E060E070E08A019B0104C00D
:10453000000F111F221F331F8A95D2F7C901B8013E
:104540001F910F910C9427220F931F9341E050E08D
:1045500060E070E004C0440F551F661F771F8A9506
:10456000D2F78091C4039091C503A091C603B09186
:10457000C7038A019B01082B192B2A2B3B2BC9014E
:10458000B8011F910F910C9427220F931F9341E0C4
:1045900050E060E070E004C0440F551F661F771FB5
:1045A0008A95D2F740955095609570958091C40397
:1045B0009091C503A091C603B091C7038A019B01E6
:1045C000082319232A233B23C901B8011F910F9106
:1045D0000C9427220F931F9341E050E060E070E0BD
:1045E00004C0440F551F661F771F8A95D2F780912C
:1045F000C4039091C503A091C603B091C7038A017B
:104600009B01082719272A273B27C901B8011F91B9
:104610000F910C9427220F931F930091C4031091C4
:10462000C5032091C6033091C703602B712B822BE9
:10463000932B1F910F910C9427220F931F9300919E
:10464000C4031091C5032091C6033091C7036023B2
:104650007123822393231F910F910C9427220F9390
:104660001F930091C4031091C5032091C60330919C
:10467000C70360277127822793271F910F910C94FE
:10468000272208958F929F92AF92BF92DF92EF926E
:10469000FF920F931F93CF93DF9300D000D01F9210
:1046A000CDB7DEB76B837C838D838A018C819D813E
:1046B000892B21F01F3F29F44F3F19F480E090E04F
:1046C0004CC08B818823C9F18090C8039090C903A6
:1046D000A090CA03B090CB038091C4039091C5030E
:1046E000A091C603B091C703882A992AAA2ABB2A97
:1046F0008FE1E82EF12CD501C4010E2C04C0B69533
:10470000A795979587950A94D2F780FF07C0DE2C6E
:10471000B8018E2D0E94FB25019729F481E0E81A4B
:10472000F10848F7D12C88E0189FF0011124E00F20
:10473000F11DEC5BFC4FD08209C088E0189FF001AE
:104740001124E00FF11DEC5BFC4FD08009831A832C
:1047500069817A818D2D0E94FB250F900F900F901B
:104760000F900F90DF91CF911F910F91FF90EF90DD
:10477000DF90BF90AF909F908F900895209121017E
:1047800030912201F90132969FEF40E05191581784
:1047900089F09F3F19F4511101C0942F4F5F4630AB
:1047A000A9F79F3F39F0F901E90FF11D97FDFA953F
:1047B0008283089508952091210130912201F90109
:1047C0003296285F3F4F9081981301C01082319636
:1047D000E217F307C1F7089581E090E0E09121012D
:1047E000F0912201E80FF91F10820196883091059F
:1047F000A9F708958091D80308959091D803892B43
:104800008093D803089580959091D803892380934D
:10481000D80308958093D80308951092D80308957B
:104820009091D703892B8093D70308958095909119
:10483000D70389238093D70308951092D70308954F
:104840008093CE030E9438259093CD038093CC03B0
:1048500008951092CE031092CD031092CC030895C8
:104860008091210190912201FC0131969C01285FE9
:104870003F4F80E0919191118F5FE217F307D1F7DD
:104880000895E0912101F09122018091D803808365
:10489000E0912101F091220190818091D703892B31
:1048A00080838091CE038823D9F10E9438252091FE
:1048B000CC033091CD038217930748F00E9438252E
:1048C0002091CC033091CD03821B930B0AC00E9430
:1048D00038252091CC033091CD0320953095820F5F
:1048E000931F8C32914070F08091D90380FF08C0F3
:1048F0008AEC96E09F938F930E949A070F900F90F7
:104900000E942924E0912101F0912201908180915F
:10491000CE03892B80830E94302481110E94292498
:1049200080912101909122010C941E1890939B017B
:1049300080939A0108958295982F9C7C392F369503
:104940003695282F237344E0249FC0011124932F10
:10495000982B292F2A7A2695892F8575880F822BE7
:1049600008950895CF93DF9300D000D01F92CDB764
:10497000DEB70F900F900F900F900F90DF91CF91B7
:104980000895089508950C949D198091EE03843044
:1049900021F11092DA0320E488E190E00FB6F89458
:1049A000A895809360000FBE2093600083B7817F3D
:1049B000846083BF83B7816083BF7894889583B711
:1049C0008E7F83BF0FB6F894A895809160008861B0
:1049D00080936000109260000FBE0895CF930E94F4
:1049E000CA080E94E1070E94CC08C0E08C2F0E94F8
:1049F000C108811104C0CF5FC031C1F701C081E09F
:104A0000CF9108950E949F190C94011E1F920F923E
:104A10000FB60F9211248F939F93AF93BF93809102
:104A2000DA03811113C08091DB039091DC03A09124
:104A3000DD03B091DE034196A11DB11D8093DB0320
:104A40009093DC03A093DD03B093DE03BF91AF919D
:104A50009F918F910F900FBE0F901F90189582E03D
:104A600084BD93E095BD9AEF97BD80936E00089545
:104A70002FB7F8948091DB039091DC03A091DD03C4
:104A8000B091DE032FBF08952FB7F8946091DB0338
:104A90007091DC038091DD039091DE032FBF0895B8
:104AA000CF92DF92EF92FF920F931F932FB7F8945C
:104AB0004091DB035091DC036091DD037091DE03D4
:104AC0002FBF6A017B01EE24FF248C0120E030E03F
:104AD000C016D106E206F30610F4415051099A01BE
:104AE000281B390BC9011F910F91FF90EF90DF90A8
:104AF000CF900895CF92DF92EF92FF920F931F9382
:104B00002FB7F894C090DB03D090DC03E090DD0376
:104B1000F090DE032FBF97018601061B170B280BB1
:104B2000390BC616D706E806F90618F0C901B80110
:104B300006C0C901B80161507109810991091F912D
:104B40000F91FF90EF90DF90CF9008951F920F92FA
:104B50000FB60F9211248F939F93AF93BF938091C1
:104B6000DB039091DC03A091DD03B091DE0301969D
:104B7000A11DB11D8093DB039093DC03A093DD03A3
:104B8000B093DE03BF91AF919F918F910F900FBEB5
:104B90000F901F9018950E942615F8942FEF87EA22
:104BA00091E6215080409040E1F700C0000087E08E
:104BB00090EBDC018093F7039093F803A093F90343
:104BC000B093FA039CE088E10FB6F894A89580931F
:104BD00060000FBE90936000FFCF28E0929FF0012D
:104BE0001124E80FF11DEE58FE4F9491892F8F701C
:104BF00092959F700895CF93C82FCB010E94ED2509
:104C0000282F30E080E1989FA0011124422B532BE4
:104C10004038510519F480E090E015C09770E92FF5
:104C2000F0E088E0C89FE00DF11D112484E0EE0F54
:104C3000FF1F8A95E1F7E20FF31FEE0FFF1FE05011
:104C4000F84985919491CF91089580E090E008957E
:104C500008958091E10380FF0BC06091260185E0FB
:104C6000689FB001112475956795759567952BC060
:104C700081FF09C06091260185E0689FB001112481
:104C80007595679520C082FF07C06091260185E079
:104C9000689FB001112417C09091E2039923D1F0CD
:104CA00060912501961788F72091260185E0289FBD
:104CB00090011124929FA001939F500D112470E048
:104CC000CA010E94F12D6038710540F4611571052B
:104CD00039F002C065E070E0862F08958FE70895EF
:104CE00081E008958091E10380FF08C06091240174
:104CF00070E0759567957595679521C081FF06C031
:104D00006091240170E07595679519C082FF04C019
:104D10006091240170E010C09091E2039923C1F0EA
:104D2000609123019617A0F780912401899FC0010B
:104D3000112470E00E94F12D6038710528F461158E
:104D4000710521F0862F08958FE7089581E0089579
:104D500061E070E0F4CF803F21F40E942926819524
:104D600004C0813F29F40E9429268093E503089519
:104D7000823F21F40E942926819504C0833F29F4B3
:104D80000E9429268093E4030895893F19F40E9424
:104D9000722605C08A3F31F40E9472268195809365
:104DA000E60308958B3F21F40E947226819504C08A
:104DB0008C3F29F40E9472268093E7030895843F74
:104DC00021F48091E303816017C0853F21F4809135
:104DD000E303826011C0863F21F48091E303846085
:104DE0000BC0873F21F48091E303886005C0883FB2
:104DF00031F48091E30380618093E30308958D3F54
:104E000021F48091E10381600BC08E3F21F48091F9
:104E1000E103826005C08F3F29F48091E103846043
:104E20008093E1030895803F39F48091E50387FF83
:104E30006CC01092E50369C0813F29F48091E503BD
:104E40001816BCF362C09091E403823F29F497FFE7
:104E50005CC01092E40359C0833F19F41916CCF3D7
:104E600054C0893F41F48091E60318160CF04DC000
:104E70001092E6034AC08A3F29F48091E60387FF37
:104E800044C0F6CF8B3F39F48091E70387FF3DC0E4
:104E90001092E7033AC08C3F29F48091E70318167B
:104EA000BCF333C0843F21F48091E3038E7F17C0AD
:104EB000853F21F48091E3038D7F11C0863F21F46B
:104EC0008091E3038B7F0BC0873F21F48091E30344
:104ED000877F05C0883F31F48091E3038F7E809304
:104EE000E30313C08D3F21F48091E1038E7F0BC05B
:104EF0008E3F21F48091E1038D7F05C08F3F29F41F
:104F00008091E1038B7F8093E1038091E403811121
:104F10000EC08091E50381110AC08091E6038111E2
:104F200006C08091E703811102C01092E203089548
:104F30008091D90383FF7EC083E097E00E94010740
:104F40008091E3031F928F938EEF96E09F938F9350
:104F50000E949A078CEF96E00E9401078091E4037B
:104F6000282F082E000C330B3F938F9389EF96E088
:104F70009F938F930E949A0787EF96E00E94010704
:104F80008091E503282F082E000C330B3F938F935D
:104F900084EF96E09F938F930E949A0782EF96E0AA
:104FA0000E9401078091E603282F082E000C330B86
:104FB0003F938F938FEE96E09F938F930E949A0773
:104FC0008DEE96E00E9401078091E703282F082EBE
:104FD000000C330B3F938F938AEE96E09F938F9351
:104FE0000E949A0787EE96E00E9401078091E203F3
:104FF0001F928F9384EE96E09F938F930E949A075F
:1050000082EE96E00E9401078091E1031F928F9348
:105010008FED96E09F938F930E949A078CED96E018
:105020000E9401078DB79EB74C960FB6F8949EBFAD
:105030000FBE8DBF83EE93E00E9467180E94382553
:105040009093E0038093DF0308951F93CF93DF9342
:105050008091DF039091E0030E945025AC01909174
:10506000E203992321F02091270130E006C020912E
:1050700028018AE0289F900111244217530708F461
:1050800085C08091E403C091E503D091E6031091BF
:10509000E703811107C0C11175C0D11173C011118F
:1050A00071C074C09F3F19F09F5F9093E203181680
:1050B00024F40E9429268093E4038091E40387FF6F
:1050C00005C00E94292681958093E4031C1624F4D0
:1050D0000E9429268093E5038091E50387FF05C0A0
:1050E0000E94292681958093E5036091E40366235D
:1050F00031F1C091E503CC2311F1062E000C770BA2
:10510000880B990B0E94D82C23E333E343E35FE33E
:105110000E943C2D0E94A02C6093E4036C2FCC0FC6
:10512000770B880B990B0E94D82C23E333E343E3DE
:105130005FE30E943C2D0E94A02C6093E5031D16A6
:1051400024F40E9472268093E6038091E60387FF91
:1051500005C00E94722681958093E603111624F4FF
:105160000E9472268093E7038091E70387FF05C0C2
:105170000E94722681958093E703DF91CF911F9162
:105180000C9498279F3F09F08FCF97CFDF91CF9155
:105190001F910895E3EEF3E085E0DF011D928A950B
:1051A000E9F71092E2031092E103089586E299E094
:1051B0000E9401071F9281E08F931F9285E08F93D9
:1051C00088ED98E09F938F930E949A070F900F901D
:1051D0000F900F900F900F9008958330E9F128F40D
:1051E000813061F0823009F10895853009F462C0A0
:1051F00008F449C0863009F474C0089580912801EC
:10520000262F30E0280F311D2F3F310524F4680F81
:105210006093280103C08FEF8093280180912801BB
:105220001F928F9381E198E072C080912701262F11
:1052300030E0280F311D2F3F310524F4680F6093B3
:10524000270103C08FEF80932701809127011F92D0
:105250008F938FEF97E05BC080912601262F30E07F
:10526000280F311D2F3F310524F4680F609326016C
:1052700003C08FEF80932601809126011F928F93A8
:105280008CEE97E044C080912501262F30E0280F56
:10529000311D2F3F310524F4680F6093250103C0B1
:1052A0008FEF80932501809125011F928F9387EDC9
:1052B00097E02DC080912401262F30E0280F311D6A
:1052C0002F3F310524F4680F6093240103C08FEF52
:1052D00080932401809124011F928F938EEB97E09D
:1052E00016C080912301262F30E0280F311D2F3F5B
:1052F000310524F4680F6093230103C08FEF80937E
:105300002301809123011F928F9383EA97E09F935B
:105310008F930E949A070F900F900F900F9008950F
:10532000833081F128F4813059F08230D1F0089532
:10533000853009F449C0B8F1863009F456C00895A3
:1053400080912801681720F4861B8093280102C0F1
:1053500010922801809128011F928F9384E997E091
:1053600054C080912701681720F4861B8093270181
:1053700002C010922701809127011F928F9382E82B
:1053800097E043C080912601681720F4861B809324
:10539000260102C010922601809126011F928F9350
:1053A0008FE697E032C080912501681720F4861BB4
:1053B0008093250102C010922501809125011F9242
:1053C0008F938AE597E021C080912401681720F42B
:1053D000861B8093240102C0109224018091240135
:1053E0001F928F9381E497E010C08091230168178A
:1053F00020F4861B8093230102C010922301809128
:1054000023011F928F9386E297E09F938F930E94D0
:105410009A070F900F900F900F900895CF93C82F79
:105420001F928F938BE29AE09F938F930E949A072B
:1054300081E090E0A0E0B0E0BC01CD0104C0660FC7
:10544000771F881F991FCA95D2F70E9432220F90AA
:105450000F900F900F90CF910C94011ECF93873235
:1054600088F58E3108F00BC18E3009F487C0D8F46E
:10547000873009F460C08B3009F44FC0863009F0E2
:1054800002C18091D903817F8E7F8093D90380E30D
:105490009AE00E94010785EE9CE00E94010781E0EE
:1054A0008093E90346C0863109F4B0C020F480310E
:1054B00009F47AC0E8C0893109F491C08B3109F44C
:1054C00049C0E1C0883349F150F4893209F4D5C0AC
:1054D000853309F4D2C0873209F0D5C0CEC08334F9
:1054E00009F4CBC028F48A3308F4CDC08953C8C06E
:1054F000883409F0C8C00E94011E84ED9CE00E941F
:1055000001072FEF83ED90E3215080409040E1F7B9
:1055100000C000000E94CB250CC087E59AE041C086
:105520008BEB9CE00E9401078091D90381608093FE
:10553000D903C1E0ADC08091D903C82FC17080FFED
:10554000EFCF87EC9CE00E9401078091D903817F17
:105550008E7F3FC09091D90391FBCC27C0F981E0A9
:10556000C827892FC0FB81F98093D903CC2319F078
:105570008EEA9CE029C080EA9CE013C09091D90398
:1055800092FBCC27C0F981E0C827892FC0FB82F9A4
:105590008093D903CC2319F081E99CE015C081E800
:1055A0009CE00E940107C5CF9091D90393FBCC27C3
:1055B000C0F981E0C827892FC0FB83F98093D90304
:1055C000CC2351F085E79CE00E9401078091D9032C
:1055D00081608093D9035CC088E69CE0E2CF89E5D6
:1055E0009CE00E9401078CE29CE00E94010785EF8D
:1055F0009BE00E94010788EC9BE00E94010783E882
:105600009BE00E94010785E59BE0CBCF87E49BE010
:105610000E9401070E9412181F928F938DE29BE057
:105620009F938F930E949A07809120011F928F93DE
:1056300086E19BE09F938F930E949A078091F402EA
:105640001F928F9383E09BE09F938F930E949A0712
:105650000E9444259F938F937F936F938CEE9AE0E3
:105660009F938F930E949A078DB79EB742960FB66D
:10567000F8949EBF0FBE8DBF5CCF80E001C08D51FE
:105680000E940E2A56CF8AEE9AE00E940107C0E0DF
:105690008C2FCF910895CF93C82F8091E90381304B
:1056A00071F020F0823009F44BC042C1E091210139
:1056B000F09122018081823209F03CC107C0E09163
:1056C0002101F09122018081823261F48C2F0E94AD
:1056D000010C811104C08C2F0E942E2A2FC081E062
:1056E00090E02CC08C2F0E942E0E811126C0C43158
:1056F000E1F070F4CB3081F0C031D1F40E94D628B3
:1057000083E29AE00E94010782E08093E90315C0DA
:10571000C93259F0C83361F480E39AE00E9401076E
:1057200087E29AE00E94010708C01092E90304C1D1
:1057300081E29AE00E940107FFC081E08170FEC013
:10574000C43228F5CE3108F0C1C0CB30A1F1D0F47D
:10575000C73009F0D3C08EE18093280182E38093A3
:1057600027018AE08093260184E18093250188E067
:105770008093240188E28093230187EC98E00E94C3
:105780000107BFC0C33149F1C431C1F0B7C0CB3448
:1057900009F4A9C028F4C93289F0C83361F0AEC059
:1057A000C13509F49EC0C23509F499C0CE3409F060
:1057B000A5C06AE09EC00E94D628A3C08091E803DD
:1057C000882319F01092E8039CC084ED98E00E94B1
:1057D000010781E08093E903B1C08EEA98E00E945E
:1057E00001078CE998E00E940107809128011F922F
:1057F0008F9389E998E09F938F930E949A0787E996
:1058000098E00E94010785E898E00E9401078091D6
:1058100027011F928F9382E898E09F938F930E94B5
:105820009A0780E898E00E94010781E798E00E94CB
:105830000107809126011F928F938EE698E09F9337
:105840008F930E949A078CE698E00E9401078BE5EF
:1058500098E00E940107809125011F928F9388E5AF
:1058600098E09F938F930E949A0786E598E00E94A4
:10587000010781E498E00E940107809124011F92B2
:105880008F938EE398E09F938F930E949A078CE307
:1058900098E00E94010785E298E00E94010780914C
:1058A00023011F928F9382E298E09F938F930E942F
:1058B0009A0780E298E00E9401078DB79EB748964C
:1058C0000FB6F8949EBF0FBE8DBF1BC0CE51EC2FFC
:1058D000F0E0E057FE4F80818093E80312C061E062
:1058E00003C061E006C06AE08091E8030E94ED28F1
:1058F00008C08091E8030E94902903C085EC98E0DD
:1059000013C08091E803882369F01F928F938FEB77
:1059100098E09F938F930E949A070F900F900F909B
:105920000F9004C08CEB98E00E94010781E006C054
:105930001092E90380E002C080E000CFCF9108958B
:105940000E94A72C6894B1110C94362D08950E94E2
:105950001B2D88F09F5798F0B92F9927B751B0F0B9
:10596000E1F0660F771F881F991F1AF0BA95C9F7E3
:1059700014C0B13091F00E94352DB1E008950C941F
:10598000352D672F782F8827B85F39F0B93FCCF3D2
:10599000869577956795B395D9F73EF49095809560
:1059A000709561957F4F8F4F9F4F0895E89409C080
:1059B00097FB3EF490958095709561957F4F8F4F42
:1059C0009F4F9923A9F0F92F96E9BB279395F69558
:1059D000879577956795B795F111F8CFFAF4BB0FD6
:1059E00011F460FF1BC06F5F7F4F8F4F9F4F16C03A
:1059F000882311F096E911C0772321F09EE8872FC4
:105A0000762F05C0662371F096E8862F70E060E07F
:105A10002AF09A95660F771F881FDAF7880F9695F8
:105A2000879597F9089557FD9058440F551F59F0E1
:105A30005F3F71F04795880F97FB991F61F09F3F7B
:105A400079F087950895121613061406551FF2CFA4
:105A50004695F1DF08C0161617061806991FF1CFF4
:105A600086957105610508940895E894BB2766271B
:105A70007727CB0197F908950E944F2D0C94C02DE4
:105A80000E94B22D38F00E94B92D20F0952311F01C
:105A90000C94A92D0C94AF2D11240C94362D0E943A
:105AA000132D70F3959FC1F3950F50E0551F629F22
:105AB000F001729FBB27F00DB11D639FAA27F00D67
:105AC000B11DAA1F649F6627B00DA11D661F829F8E
:105AD0002227B00DA11D621F739FB00DA11D621F73
:105AE000839FA00D611D221F749F3327A00D611D90
:105AF000231F849F600D211D822F762F6A2F112472
:105B00009F5750409AF0F1F088234AF0EE0FFF1FA4
:105B1000BB1F661F771F881F91505040A9F79E3FFB
:105B2000510580F00C94A92D0C94362D5F3FE4F3C1
:105B3000983ED4F3869577956795B795F795E79551
:105B40009F5FC1F7FE2B880F911D9695879597F95A
:105B5000089597F99F6780E870E060E008959FEFEF
:105B600080EC089500240A941616170618060906F4
:105B7000089500240A9412161306140605060895C3
:105B8000092E0394000C11F4882352F0BB0F40F44B
:105B9000BF2B11F460FF04C06F5F7F4F8F4F9F4F8B
:105BA0000895991B79E004C0991F961708F0961B79
:105BB000881F7A95C9F780950895AA1BBB1B51E1F0
:105BC00007C0AA1FBB1FA617B70710F0A61BB70B6D
:105BD000881F991F5A95A9F780959095BC01CD0112
:105BE000089597FB072E16F4009407D077FD09D08F
:105BF0000E94DD2D07FC05D03EF4909581959F4FC6
:105C00000895709561957F4F0895A1E21A2EAA1B01
:105C1000BB1BFD010DC0AA1FBB1FEE1FFF1FA2175C
:105C2000B307E407F50720F0A21BB30BE40BF50B59
:105C3000661F771F881F991F1A9469F760957095E2
:105C4000809590959B01AC01BD01CF010895EE0FA9
:0E5C5000FF1F0590F491E02D0994F894FFCF0A
:105C5E00560959095A095B095C095209D609BC094A
:105C6E0055095D090A01CB10BC119911651131114D
:105C7E0001CF032808140A321E524E2D3432004C26
:105C8E00554641004F4646004F4E00434F4E4E0084
:105C9E00506F776572656400556E617474616368E8
:105CAE0065640044656661756C7400416464726578
:105CBE007373656400436F6E666967757265640021
:105CCE003F0053757370656E64656400404D3622F7
:105CDE003206E505AF058D05190532054B05640540
:0A5CEE00010203040506070809007F
:1068000088000000000000000400050006000700EA
:10681000080009000A000B000C000D000E000F001C
:1068200010001100120013001400150016001700CC
:10683000180019001A001B001C001D001E001F007C
:10684000200021002200230024002500260027002C
:10685000280035002A002B002C002D002E002F00D0
:1068600030000000320033003400290036003700C9
:106870003800E00000000000000000000000000000
:106880000000000000000000000000000000000008
:1068900000000000000000000000000000004F00A9
:1068A00050005100520000000000000000000000F5
:1068B00000000000000000000000000000000000D8
:1068C00000000000000000000000000000000000C8
:1068D00000000000000000000000000000000000B8
:1068E0000000000000000000890087008A008B0083
:1068F000F1A1E100E200E300F1A1E500E600000003
:106900000100000000000000EA4401000100E24430
:106910000100010001005500460054004A004B00F0
:10692000560057004700480001000100E9440100FB
:106930000100010001000100010001003A003B00DC
:106940003C003D003E003F0040004100420043004B
:10695000580001004C00390001004400450052007D
:1069600001000000010050004F0081404D004E002A
:1069700051000100000000000000000000000000C5
:106980000000000000000000000000000000000007
:1069900000000000000000000000000000004D00AA
:1069A0004A004E004B000000000000000000000004
:1069B00000000000000000000000000000000000D7
:1069C00000000000000000000000000000000000C7
:1069D00000000000000000000000000000000000B7
:1069E000000000000000000049000100010001005B
:1069F0000100010001000100010001000100000090
:00000001FF
